:100000000C9463000C948B000C948B000C942909C5
:100010000C9429090C9429090C948B000C948B00E6
:100020000C948B000C948B000C948B000C94C508E2
:100030000C948B000C948B000C948B000C948B0014
:100040000C9423080C948B000C9493080C946D086A
:100050000C948B000C948B000C948B000C948B00F4
:100060000C948B000C948B0000000008000201002F
:100070000003040700000000000000000000000072
:1000800023002600290000000000240027002A0089
:1000900000000000250028002B00040404040404D0
:1000A0000404020202020202030303030303010227
:1000B00004081020408001020408102001020408F6
:1000C0001020A109A80D11241FBECFEFD8E0DEBF7C
:1000D000CDBF11E0A0E0B1E0E6E7FCE102C0059091
:1000E0000D92A832B107D9F722E0A8E2B1E001C031
:1000F0001D92A13CB207E1F710E0C2E6D0E004C0D7
:100100002197FE010E94280EC136D107C9F70E942F
:10011000100B0C942E0E0C940000DC01FB01460F1A
:10012000571FE417F507E1F021912F778D919C91EE
:100130001197822711969C938E9327E06D917C9165
:100140001197CB019695879560FF04C030EF832708
:1001500032E2932711969C938E93215079F7E1CF49
:1001600008958091BC029091BD02892B59F1E091D4
:100170009A01F0919B0182E0E23AF80719F1309779
:1001800039F0A389B4899C918589809589238C93C2
:100190008091C0028E7F8093C002109299011092CC
:1001A000980182EA92E090939B0180939A01E091FA
:1001B000B502F091B60280819091B702892B8083BD
:1001C00081E0089580E0089590E0FC01E859FF4F38
:1001D0002491FC01E255FF4F3491FC01E656FF4F9C
:1001E000E491EE23C9F0222339F0233001F1A8F481
:1001F000213019F1223029F1F0E0EE0FFF1FE05716
:10020000FF4FA591B4918FB7F894EC91611126C07E
:1002100030953E233C938FBF08952730A9F02830B6
:10022000C9F0243049F7809180008F7D03C0809110
:1002300080008F7780938000DFCF84B58F7784BD77
:10024000DBCF84B58F7DFBCF8091B0008F7780931B
:10025000B000D2CF8091B0008F7DF9CF3E2BDACFA6
:100260002FB7F89460919401709195018091960157
:10027000909197012FBF0895AF92BF92CF92DF92D6
:10028000EF92FF920F931F93CF93DF936C017B014B
:100290008B01040F151FEB015E01AE18BF08C017DC
:1002A000D10759F06991D601ED91FC910190F0814F
:1002B000E02DC6010995892B79F7C501DF91CF9112
:1002C0001F910F91FF90EF90DF90CF90BF90AF9074
:1002D0000895FC01538D448D252F30E0842F90E04C
:1002E000821B930B541710F0CF9608950197089531
:1002F000FC01918D828D981761F0A28DAE0FBF2FFA
:10030000B11D5D968C91928D9F5F9F73928F90E04F
:1003100008958FEF9FEF0895FC01918D828D9817BE
:1003200031F0828DE80FF11D858D90E008958FEFFB
:100330009FEF08950F931F930E9430016093A401D3
:100340007093A5018093A6019093A7018CE991E099
:100350000E948C0197FF1DC00E9430010091A401F2
:100360001091A5012091A6013091A701601B710B8E
:10037000820B930B0091A0011091A1012091A20189
:100380003091A3016017710782079307F8F28FEF8E
:100390009FEF1F910F910895FC01918D228D892F60
:1003A00090E0805C9F4F821B91098F73992708957D
:1003B0008CE991E00E94CC0121E0892B09F420E036
:1003C000822F089580E090E0892B29F00E94D801C7
:1003D00081110C9400000895FC01A48DA80FB92F81
:1003E000B11DA35ABF4F2C91848D90E001968F735D
:1003F0009927848FA689B7892C93A089B1898C917C
:10040000837080648C93938D848D981306C00288CA
:10041000F389E02D80818F7D80830895EF92FF9294
:100420000F931F93CF93DF93EC0181E0888F9B8D17
:100430008C8D98131AC0E889F989808185FF15C0D1
:100440009FB7F894EE89FF896083E889F9898081F4
:100450008370806480839FBF81E090E0DF91CF91C3
:100460001F910F91FF90EF900895F62E0B8D10E0E5
:100470000F5F1F4F0F731127E02E8C8D8E110CC054
:100480000FB607FCFACFE889F989808185FFF5CF9F
:10049000CE010E94EC01F1CFEB8DEC0FFD2FF11D91
:1004A000E35AFF4FF0829FB7F8940B8FEA89FB89DC
:1004B00080818062CFCFCF93DF93EC01888D88233A
:1004C000B9F0AA89BB89E889F9898C9185FD03C0B7
:1004D000808186FD0DC00FB607FCF7CF8C9185FF9C
:1004E000F2CF808185FFEDCFCE010E94EC01E9CFF4
:1004F000DF91CF91089520919A0130919B012817A7
:10050000390771F49091980180919901981741F001
:10051000E0919801F0E0E85DFE4F808190E0089561
:100520008FEF9FEF08950895EF92FF920F931F931F
:10053000CF93DF93DC015C96ED90FC905D97E11426
:10054000F10479F481E090E013969C938E931297D6
:1005500090E080E0DF91CF911F910F91FF90EF909D
:1005600008955196ED91FC91529750968C91509729
:10057000982F90950FB75E962C915E97122F127060
:1005800021FD6095F8942081112319F1282B2083F7
:10059000E7012197F1F728E0462F50E0308160FF16
:1005A0001AC0382B3083E7012197F1F7BA0175950E
:1005B0006795215089F7112381F0808189238083F9
:1005C0000FBF5C968D919C910197F1F781E090E0CF
:1005D000C1CF2923DCCF3923E5CF9081892BEFCF01
:1005E00020919A0130919B012817390771F480916D
:1005F00099012091980190E0805C9F4F821B9109A6
:1006000060E470E00E94000E089590E080E008959C
:1006100020919A0130919B0128173907B9F49091E4
:10062000980180919901981789F0E0919801F0E084
:10063000E85DFE4F80812091980130E02F5F3F4FB1
:100640002F7333272093980190E008958FEF9FEF49
:10065000089590E080E00895CF93DF93EC010E942D
:100660003001688379838A839B83DF91CF910895DA
:10067000FC0110821582148213821282118216826A
:100680001782108611860895DC01ED91FC91119777
:1006900012968D919C911397E817F90739F0819183
:1006A000ED93FC93FB01808381E0089580E0089541
:1006B000CF93DF93EC01DB01ED91FC911197309723
:1006C000D1F012964D915D916D917C911597858534
:1006D0009685A785B089481759076A077B0759F49B
:1006E0008AE07596DE0101900D928A95E1F7CE01C0
:1006F000DF91CF910895CE010E94380381E0888375
:100700008A838FEF9FEFDC018E839F83A887B98751
:10071000EECFCF92DF92EF92FF920F931F93CF9382
:10072000DF9300D0CDB7DEB77C01FC01608341834D
:100730000283F901DC011396200F311FE217F30742
:1007400019F081918D93FACFA8014D5F5F4F67013A
:10075000C40ED51E8FEF9FE39A838983B701CE0124
:1007600001960E948D0089819A818095FFE39F27E1
:10077000282F2F77F6012083F701E00FF11F880F54
:10078000892F881F990B91958F778483C8010596CF
:100790000F900F90DF91CF911F910F91FF90EF90ED
:1007A000DF90CF900895EF92FF920F931F93CF9316
:1007B000DF93CDB7DEB7EF970FB6F894DEBF0FBE6D
:1007C000CDBFE0915B02F0915C02E3A0F4A0209128
:1007D0005D022DA322E030E03CA32BA34EA346FFF5
:1007E00007C020917A0243E050E05CA34BA32FA303
:1007F000DB0112960D911C912BA13CA1FB013496BB
:10080000DE01A20FB31F9596B8016E0F7F1F6E1702
:100810007F0719F041914D93FACF020F131F1CA3CC
:100820000BA39E012B5D3F4FAC0160915E02CE0198
:1008300001960E948903D701ED91FC910280F3811A
:10084000E02DAC01BE016F5F7F4FC7010995EF96A8
:100850000FB6F894DEBF0FBECDBFDF91CF911F91D1
:100860000F91FF90EF9008952F923F924F925F92D9
:100870006F927F928F929F92AF92BF92CF92DF92B0
:10088000EF92FF920F931F93CF93DF93CDB7DEB715
:10089000CC54D1090FB6F894DEBF0FBECDBF6C01AA
:1008A0007B01742E49012B961FAF0EAF2B97FB01D6
:1008B00084819581A681B78128968CAF9DAFAEAF1C
:1008C000BFAF2897CE01805C9F4F0E942C032896D3
:1008D0008CAD9DADAEADBFAD2897B7FD12C00E94E7
:1008E000300128960CAD1DAD2EAD3FAD2897601B95
:1008F000710B820B930B24966CAF7DAF8EAF9FAFC5
:100900002497C40180612D969FAF8EAF2D9734E060
:10091000232E312C6624639444244A944FE3542EAE
:100920002B96EEADFFAD2B9784819581A681B78183
:10093000B7FD44C00E9430012B96AEADBFAD2B97E2
:100940000D911D912D913C911397601B710B820BA2
:10095000930B14960D911D912D913C911797601753
:1009600071078207930750F1C6010E94380381E0A6
:10097000F601808382838EEF9FEFAFEFBFEF868318
:100980009783A087B187C601C45BDF4F0FB6F89489
:10099000DEBF0FBECDBFDF91CF911F910F91FF90B2
:1009A000EF90DF90CF90BF90AF909F908F907F900F
:1009B0006F905F904F903F902F90089528968CAD48
:1009C0009DADAEADBFAD2897B7FD4DC00E943001C3
:1009D00024960CAD1DAD2EAD3FAD2497601B710B61
:1009E000820B930B28960CAD1DAD2EAD3FAD289715
:1009F0006017710782079307B0F1CE01805C9F4FAB
:100A00000E942C03D7011C968C918F5F87FD81E09B
:100A1000F701848792819DA32C96FFAD2C97FEA3AE
:100A20008FA33CA22BA278A6D701ED91FC91119740
:100A300083A094A004E010E09E012B5D3F4F43E2B1
:100A400050E013966C91CE0101960E948903D40167
:100A5000ED91FC910280F381E02DAC01BE016F5F4E
:100A60007F4FC4010995F701008111814801F3E02E
:100A70008F0E911CD80193968D919C91DC01ED9184
:100A8000FC910284F385E02D099597FD49CF87FD00
:100A900004C0F8012281222331F0D80111961C9262
:100AA0001E9212961C92F80120813181203231056C
:100AB00050F4A9014F5F5F4F51834083200F311FD6
:100AC000D90113968C93F80140815181453051052D
:100AD000C0F0838187FF15C02581CA0105972817BB
:100AE000190679F45A824982B401CE0101960E9416
:100AF0008D0089819A8181389F4019F4D80112961E
:100B00006C92F8018281882309F4B4CFD701ED916A
:100B1000FC911197938113968C91981301CF848146
:100B2000833409F0FDCE00811181055011094F0178
:100B300026E0820E911CCE0101960E9438039AA2F3
:100B400089A2080D191D1CA30BA3BE016E5F7F4F68
:100B5000CE0181960E944403882309F47BC0BE0124
:100B60006D5F7F4FCE0181960E944403882309F474
:100B700071C08B8184FD65C08B8186FD70C0BE0114
:100B80006A5F7F4FCE0181960E944403882309F457
:100B900061C010E000E0812C912C5401BE01685B23
:100BA0007F4FCE0181960E9444038823D9F0299675
:100BB0002FAD2997822F8F7390E0B0E0A0E0002E38
:100BC00004C0880F991FAA1FBB1F0A94D2F7882A56
:100BD000992AAA2ABB2A26FF05C00A5F1F4F0E3199
:100BE0001105E1F6D501C401B695A79597958795AE
:100BF00080FE07C0B095A095909581959F4FAF4F0F
:100C0000BF4F8F839887A987BA872B8120FF05C0A4
:100C1000181619061A061B06ECF4698289818823C6
:100C200009F47ECED7011C969C918C81981378CEC6
:100C30008AE0FE013196D60101900D928A95E1F786
:100C4000A2CEBE016C5F7F4FCE0181960E9444030D
:100C5000811192CFCE0101960E943803DFCFBE01F1
:100C60006B5F7F4FCE0181960E944403811187CF35
:100C7000F1CFEF92FF920F931F93CF93DF93CDB7F6
:100C8000DEB72A970FB6F894DEBF0FBECDBF7B014B
:100C90008C0120E430E041E050E06BE572E0CE01F1
:100CA00001960E9434048AE0FE013196D70101903A
:100CB0000D928A95E1F7F701828180FF04C0868159
:100CC000978197FD15C0F701848180937A0281E0B6
:100CD00080937B0280E02A960FB6F894DEBF0FBEA9
:100CE000CDBFDF91CF911F910F91FF90EF900895AD
:100CF00081E0F1CFDF92EF92FF920F931F93CF939A
:100D0000DF93CDB7DEB72A970FB6F894DEBF0FBEDC
:100D1000CDBF7C01D42EFC012389348941895289BD
:100D20008B01BC01CE0101960E9434048AE0FE01D1
:100D30003196D701559601900D928A95E1F7F7010A
:100D4000878980FF04C0838D948D97FD16C0F701BD
:100D5000818D978D891789F0811111C08D2D2A966B
:100D60000FB6F894DEBF0FBECDBFDF91CF911F91BC
:100D70000F91FF90EF90DF90089581E0F0CF80E039
:100D8000EECF8F929F92AF92BF92CF92DF92EF926F
:100D9000FF920F931F93CF93DF93CDB7DEB72897C2
:100DA0000FB6F894DEBF0FBECDBF7C016B018A0188
:100DB0008090680290906902A0906A02B0906B02E5
:100DC0008FEF881A980AA80AB80A8092680290924F
:100DD0006902A0926A02B0926B0280917C02882321
:100DE00029F1C7010E94D3032BE532E03A8329831E
:100DF0008B829C82AD82BE823A81482D5C816D815E
:100E00007E8180E090E028960FB6F894DEBF0FBE9A
:100E1000CDBFDF91CF911F910F91FF90EF90DF90A9
:100E2000CF90BF90AF909F908F9008958091630274
:100E300090916402A0916502B09166028D839E83B9
:100E4000AF83B887CE0101960E942C0380917B026C
:100E5000882311F1006481E090E090936D0280930B
:100E60006C0210936F0200936E0280917A028F5F82
:100E700087FD81E080937A02A801B601C7010E9434
:100E8000D30340E0BE016F5F7F4F8BE592E00E948D
:100E90007A06882389F3A8CF60E772E0CE01019635
:100EA0000E9439068111A0CFD5CF8F929F92AF9229
:100EB000BF92EF92FF920F931F93CF93DF93CDB723
:100EC000DEB72A970FB6F894DEBF0FBECDBF8C01F8
:100ED0007B01B801CE0101960E9458038B8181FFEE
:100EE0001AC0F80180819181009799F382809380E4
:100EF000A480B580FC014585568567857089841678
:100F00009506A606B70629F741E0B7010E947A06C2
:100F1000882339F3DECF86E0F801DE0111960190D7
:100F20000D928A95E1F729813A814B815C816D812F
:100F30007E8180E090E02A960FB6F894DEBF0FBE67
:100F4000CDBFDF91CF911F910F91FF90EF90BF9098
:100F5000AF909F908F9008958F929F92AF92BF9283
:100F60000F931F93CF93DF93CDB7DEB7A1970FB643
:100F7000F894DEBF0FBECDBF19A2423008F44AE09C
:100F80008E010F5D1F4F842E912CB12CA12CA50139
:100F900094010E94CF0DE62FB901CA01EA3044F551
:100FA000E05DD801EE938D01232B242B252B79F7BF
:100FB00090E080E0109769F0FD0101900020E9F7D2
:100FC0003197AF014A1B5B0BBD018CE991E00E9498
:100FD0003C01A1960FB6F894DEBF0FBECDBFDF91E6
:100FE000CF911F910F91BF90AF909F908F900895D8
:100FF000E95CD7CFCF92DF92EF92FF92CF93DF934E
:101000006B017C016DE28CE991E00E940E02EC0123
:1010100066277727CB016C197D098E099F094AE065
:101020000E94AC078C0F9D1FDF91CF91FF90EF9036
:10103000DF90CF90089542E050E064E271E08CE9E7
:1010400091E00C943C011F920F920FB60F92112465
:101050002F933F938F939F93AF93BF93809194016E
:1010600090919501A0919601B091970130919301D3
:1010700023E0230F2D3758F50196A11DB11D2093B4
:1010800093018093940190939501A0939601B0935E
:10109000970180918F0190919001A0919101B09161
:1010A00092010196A11DB11D80938F019093900133
:1010B000A0939101B0939201BF91AF919F918F91B5
:1010C0003F912F910F900FBE0F901F90189526E81B
:1010D000230F0296A11DB11DD2CF1F920F920FB602
:1010E0000F9211242F933F934F935F936F937F93AE
:1010F0008F939F93AF93BF93EF93FF938CE991E00E
:101100000E94EC01FF91EF91BF91AF919F918F9160
:101110007F916F915F914F913F912F910F900FBEF3
:101120000F901F9018951F920F920FB60F921124D7
:101130002F938F939F93EF93FF93E091AC01F091E6
:10114000AD018081E091B201F091B30182FD1BC03D
:1011500090818091B5018F5F8F732091B6018217C6
:1011600041F0E091B501F0E0E456FE4F958F809399
:10117000B501FF91EF919F918F912F910F900FBE2D
:101180000F901F9018958081F4CF1F920F920FB689
:101190000F9211242F933F938F939F93EF93FF937D
:1011A00080918C0187FF1FC01092850010928400EF
:1011B00080918C018F5F80938C0180918C0187FFDF
:1011C00004C080918C018C30ACF0809184009091AF
:1011D0008500049680349C4990F180918400909120
:1011E000850004962EC080918C0187FFE1CF80910D
:1011F0008C01DECF2091840030918500E0918C013C
:101200008E2FEE0F990BFC01EE0FFF1FE80FF91F59
:10121000E859FE4F81819281820F931F909389003C
:101220008093880080918C01FF91EF919F918F9125
:101230003F912F910F900FBE0F901F90189580E453
:101240009CE990938900809388008FEF80938C01B4
:10125000EBCF1F920F920FB60F9211242F933F9353
:101260004F935F936F937F938F939F93AF93BF93AE
:10127000EF93FF93E0919A01F0919B01309749F031
:10128000A685B7858585968D91FF14C09C9189238D
:10129000A1F4FF91EF91BF91AF919F918F917F91B9
:1012A0006F915F914F913F912F910F900FBE0F90D3
:1012B0001F9018959C91892361F7A389B4899C910B
:1012C0008589809589238C93868997890197F1F781
:1012D000608D718DA685B785558538E020E0CB01FE
:1012E0000197F1F7822F90E095958795282F4C91E3
:1012F000452309F02068315091F7868D81FD2095B6
:101300008091990190E001968F739927309198010F
:10131000381799F0A0919901B0E0A85DBE4F2C93C9
:1013200080939901828D938D0197F1F7A389B489F8
:101330008C919589892B8C93ACCF868D8160868F1B
:10134000F1CF8F929F92AF92BF92CF92DF92EF92A6
:10135000FF920F931F93CF93DF9310929F011092F0
:101360009E0188EE93E0A0E0B0E08093A00190930E
:10137000A101A093A201B093A30124E031E0309336
:101380009D0120939C0125EC30E03093A90120932E
:10139000A80124EC30E03093AB012093AA0120ECAB
:1013A00030E03093AD012093AC0121EC30E030937C
:1013B000AF012093AE0122EC30E03093B1012093D5
:1013C000B00126EC30E03093B3012093B2011092CB
:1013D000B5011092B6011092B7011092B8011092A7
:1013E000A5021092A4028093A6029093A702A09354
:1013F000A802B093A90286E191E09093A3028093A2
:10140000A2021092B9021092B8021092BB0210927E
:10141000BA021092BD021092BC021092BF0210924A
:10142000BE026091C0026E7F6D7F6093C0026695C0
:10143000617081E068278BE00E94E40049EB50E096
:10144000FA01649185EA90E0FC012491222399F04D
:1014500030E0220F331FF901EA57FF4FA591B491F5
:10146000F901E057FF4F259134912FB7F8943C9143
:10147000632B6C932FBFFA0144914093B202FC019D
:101480008491E82FF0E0EE0FFF1FE057FF4F8591AA
:1014900094919093B4028093B30208EB10E0F801AA
:1014A0002491C4EAD0E0FE0184918823C9F090E041
:1014B000880F991FFC01EA57FF4FA591B491FC01D9
:1014C000E057FF4F459154913FB7F8949C91822F7C
:1014D000809598239C93FA019081892380833FBF54
:1014E0008091C00281FD04C061E08AE00E94E400B6
:1014F0008AE08093AE02F80104910093AF02FE01EE
:10150000C491EC2FF0E0EE0FFF1FE458FF4F8591E0
:1015100094919093B1028093B002CDE7D2E0109203
:101520007E0210927D0210927F0282EA92E09093F6
:10153000A1028093A002D0935C02C0935B02109240
:101540005D0210E810935E0210926702109268022A
:101550001092690210926A0210926B0280E792E088
:101560000E94380310927A0210927B0281E38093EA
:101570005D0294E6892E912CA12CB12C80925F0201
:1015800090926002A0926102B0926202CC24CA944E
:10159000DC2C7601C0926302D0926402E092650274
:1015A000F092660210927C02D0933A02C093390204
:1015B00010923B0210933C02109245021092460298
:1015C0001092470210924802109249028EE492E073
:1015D0000E943803109258021092590282E38093BD
:1015E0003B0280923D0290923E02A0923F02B09256
:1015F0004002C0924102D0924202E0924302F09235
:10160000440210925A02DF91CF911F910F91FF90E7
:10161000EF90DF90CF90BF90AF909F908F90089504
:10162000CF93DF93CDB7DEB7C555D1090FB6F89488
:10163000DEBF0FBECDBF789484B5826084BD84B513
:10164000816084BD85B5826085BD85B5816085BDBD
:1016500080916E00816080936E0010928100809175
:1016600081008260809381008091810081608093FD
:101670008100809180008160809380008091B10022
:1016800084608093B1008091B00081608093B0004D
:1016900080917A00846080937A0080917A008260E1
:1016A00080937A0080917A00816080937A008091A3
:1016B0007A00806880937A001092C1001092BD0277
:1016C0001092BC021092BB021092BA021092B902A0
:1016D0001092B8028DE991E09093BF028093BE0210
:1016E0009091AE02963108F047C02DEB30E0309378
:1016F000B9022093B8022BE931E03093BB0220936A
:10170000BA022CE231E03093BD022093BC0220915A
:10171000680084E0983048F031E09E3008F430E012
:1017200081E001C0880F3A95EAF7822B8093680028
:101730002DE630E0983050F02BE630E09E3030F06F
:101740002CE630E0963110F030E020E03093B60225
:101750002093B502292F30E0983008F0C1C181E014
:1017600001C0880F9A95EAF78093B7028091BE0274
:101770009091BF020197F1F70E94B1000E94B10061
:10178000E091AC01F091AD0182E08083E091A8018D
:10179000F091A9011082E091AA01F091AB018FECC8
:1017A00080831092B401E091B001F091B10116E094
:1017B0001083E091AE01F091AF0180818061808360
:1017C000E091AE01F091AF01808188608083E0916B
:1017D000AE01F091AF01808180688083E091AE011D
:1017E000F091AF0180818F7D80831C821B8250E04D
:1017F00040E0BE016F5F7F4F80E290E00E94C10633
:101800002AA73BA74CA75DA76EA77FA7BE01665D71
:101810007F4FCE0180960E9458031C821B8250E0AD
:1018200040E0BE016F5F7F4F82E290E00E94C10600
:1018300025962FAF259726963FAF269727964FAF31
:10184000279728965FAF289729966FAF29972A96F2
:101850007FAF2A97FE01EC5BFF4FDE01A65BBF4F17
:10186000812F01900D928A95E1F7FE01E65BFF4F13
:10187000DE01909601900D921A95E1F78FEF9FEFA0
:10188000DC018D839E83AF83B887CE0101960E94D1
:101890002C03BE016F5F7F4FCE0180960E945507DB
:1018A00061962FAF619762963FAF629763964FAF95
:1018B000639764965FAF649765966FAF659766961A
:1018C0007FAF66978091630290916402A091650258
:1018D000B09166028EA79FA7A8ABB9ABCE018A963E
:1018E0000E942C03CE0101960E94380380917B0256
:1018F000811103C1BE016F5F7F4FCE018A960E94A6
:101900003906882309F4F9C06F81788589859A851D
:1019100097FF05C10E94FA070E941B0871E4B72EC9
:1019200044244A94542C320100E010E08CE991E008
:101930000E94CC01892BD1F30E949A01FC0197FDF2
:10194000FAC08D32910521F0C0970A9708F0EBC0DC
:10195000C12CD12C7601A12CE130F105D9F0ED326A
:10196000F10509F4E5C0CF01C0970A9798F4AAE001
:10197000B0E0A70196010E94C40D6F01FF0FEE08B1
:10198000FF08C60ED71EE81EF91E80E3C81AD1084C
:10199000E108F1088CE991E00E9478010E949A0127
:1019A000FC01C0970A97C0F2E130F105A9F2AA2024
:1019B00041F0F094E094D094C094C11CD11CE11C7F
:1019C000F11CD0928E01C0928D01B601DD0C880B06
:1019D000990B97FFB4C00E94FA070E941B08209140
:1019E0008D0130918E01BD82C901032E000CAA0B1E
:1019F000BB0B37FFA8C0B095A095909581959F4FE0
:101A0000AF4FBF4F880F991FAA1FBB1F8160FE01F8
:101A1000369621E030E0482F4F7350E48034910532
:101A2000A105B10508F450E02F5F3F4F452B4193CE
:101A300046E0B695A795979587954A95D1F7009773
:101A4000A105B10541F73C832B8350E040E0BE0186
:101A50006F5F7F4F84E290E00E94C10628A339A304
:101A60004AA35BA36CA37DA386E0FE01B096DE01D2
:101A70009A9601900D928A95E1F786E0FE01BA965A
:101A8000DE01D29601900D928A95E1F786E0FE0183
:101A9000F296DE01DE9601900D928A95E1F74D8275
:101AA0005E826F827886CE0101960E942C03BE0171
:101AB0006F5F7F4FCE01CE960E94550728AF39AF9A
:101AC0004AAF5BAF6CAF7DAF0115110509F42ECFA6
:101AD0000E94D801882309F429CF0E94000026CF54
:101AE0009E3040F42850310981E001C0880F2A95CA
:101AF000EAF73ACE2E503109F7CF8E01065D1F4F1F
:101B000030E020E041E050E06BE572E0CE018096ED
:101B10000E9434046EA17FA188A599A5F9CE4AE060
:101B20000E94AC07F9CE8CE991E00E94780104CFC5
:101B3000AA24A3942FCFC12CD12C760142CF4AE006
:101B40000E94AC074ACF880F991FAA1FBB1F5FCF07
:101B500086E191E09093A3028093A20280919A0182
:101B600090919B01825A924071F4E091B502F091FC
:101B7000B60290818091B70280958923808310926C
:101B80009B0110929A0108950E94F10DA59F900D5E
:101B9000B49F900DA49F800D911D11240895A1E282
:101BA0001A2EAA1BBB1BFD010DC0AA1FBB1FEE1FD7
:101BB000FF1FA217B307E407F50720F0A21BB30B22
:101BC000E40BF50B661F771F881F991F1A9469F79E
:101BD00060957095809590959B01AC01BD01CF01FA
:101BE0000895A29FB001B39FC001A39F700D811DF6
:101BF0001124911DB29F700D811D1124911D089516
:101C000097FB072E16F4009407D077FD09D00E94A9
:101C1000140E07FC05D03EF4909581959F4F0895D2
:101C2000709561957F4F0895AA1BBB1B51E107C0BA
:101C3000AA1FBB1FA617B70710F0A61BB70B881F5C
:101C4000991F5A95A9F780959095BC01CD010895EB
:101C5000EE0FFF1F0590F491E02D099410E0C2E60D
:101C6000D0E004C0FE010E94280E2196C336D107A1
:061C7000C9F7F894FFCF54
:101C7600000000000E023C0169015B02CC01780104
:101C86008C010000000094023C0129039302F0023B
:081C960008037B020D0A0000A7
:00000001FF
